:020000040000FA
:200000002020202020202020202020202020202020202020202020202020202020202020E0
:200020002020202020202020202020202020202020202020202020202020202020202020C0
:200040002020202020202020202020202020202020202020202020202020202020202020A0
:20006000202020202020202020202020202020202020202020202020202020202020202080
:00000001FF
